:020000040000FA
:02000000D02806
:08000800A82A8207000002345F
:100010000234023402340234023402340034013433
:1000200003340334033403340334033403348207C6
:10003000000020342E3420342E3420342E3420344A
:100040002E3420342E3420342E3420342E342034D8
:10005000203482070000EE34E134D434C834BD3497
:10006000B234A8349F3496348E3486347E34773458
:1000700070346A3464345E34593454344F344B34FD
:10008000473443343F343B343834353432342F34FE
:100090002C342A3427342534233421341F341D349E
:1000A0001C341A34193417341634153413341234FA
:1000B000113410340F340E34003482070000E83459
:1000C0007C34D434E4349C34F834EC3474348034E8
:1000D0000C34143490347434C0346C347434D034EC
:1000E0007C347834BC34403408340C344834BC3468
:1000F000603438343C346834C0343C34E034A034A8
:1001000084348834A434E03430349C342034B4341F
:1001100060342034F034D034C434C434D434F034B3
:100120008207000000348034013481340234033407
:1001300083340434843405348534063410349034E4
:1001400011349134123413349334143494341534F8
:10015000953416342034A0342134A134223423348D
:10016000A3342434A4342534A53426343034B034B4
:100170003134B13432343334B3343434B4343534C8
:08018000B53436344034C034BC
:1001A0008316103085008601D8308100831280309C
:1001B0008B001030A3008D018C0199019A019B01E5
:1001C0008F018E018312850186014A223D22B322CE
:1001D0001730AF220030A000252223089600051A10
:1001E000EF28051EF12881018D010B118B160230BD
:1001F0008107051AF928051EFB288B1201088C00BF
:100200009A070318990A0D08990703189B0A960B79
:10021000EF2810302302031D112903109B0C990CA9
:100220009A0C03109B0C990C9A0C1A088C00190854
:100230008D001B0891009A0199019B01BE22C822E2
:100240000510851005119108031D39290E300D0286
:10025000031C2F29FD300D02031839293E290F30C8
:10026000AB222B309622E8280F30AB223F3096226B
:10027000E8280F30AB222D309622E8285E300D02A0
:10028000031845291030A30047290830A300900126
:10029000900A1008292091009108031934298F0031
:1002A000A50010085D208E00A4000D08A7000C0812
:1002B000A600DD21FF30A200A708031D662926083D
:1002C000FC39031D6629A201C921E828031C48291D
:1002D000900310082920940010085D209500900AD2
:1002E0001408A7001508A6000F08A5000E08A40012
:1002F000DD21FA2127089300260892000F08A500A7
:100300000E08A400ED212708AA002608AC00130857
:10031000A7001208A600FA21FA21FA212708930063
:1003200026089200FE212C08A6002A08A700DD213D
:100330000318B3299B29053098000515F030A20059
:1003400090031508AD001408AB0008309100AE0111
:10035000AE0A910A11221F220318A829AE0303191D
:10036000CA211108D229043098000514A2010E08F0
:10037000AD000F08AB0007309100AE019103AE0A4B
:1003800003221F22031CBE29AE030319CA21110830
:10039000D229D22285140730AF22FF309622FF30B7
:1003A000962208009100110831020319DB29110877
:1003B000AF2218089622D222E8282408A90025088E
:1003C000A800F4212408A6070318A70A2508A707F0
:1003D0002908A4002808A50008002408A607031877
:1003E000A70A2508A7070800A409A40A0319A5035A
:1003F000A50908000310A70CA60C08000D08A5000D
:100400000C08A40008002D08A4002B08A500120861
:10041000A6001308A700ED212608AD002708AB00B1
:1004200008002D08A6002B08A7001208A400130836
:10043000A500DD212608AD002708AB0008000D0847
:10044000A5000C08A400DD2108006E30A10000000A
:1004500000000000000000000000A10B272AA00BF4
:10046000252A003408309600960B342A08008900AB
:1004700083160814831208080800403087220030D1
:10048000AE002E0837229622AE0AAE1E412A2E1E3C
:10049000412A0800FF30A0002522303086000614D3
:1004A000000006103230A0002522303068223030A3
:1004B00068222030682201308722283087220830C5
:1004C000872206308722083087220F3087220800D3
:1004D00086000614000006100A30A000252208003D
:1004E0008316F03086048312061186150614000068
:1004F00006089F00061000000614000006109F1B4F
:10050000742A861183160F308605831208009E0018
:1005100070221E08F03986000614000006101E0E18
:10052000F039860006140000061008009E007022B4
:100530001E08F039860006150614000006101E0E6F
:10054000F039860006150614000006100611080092
:100550000B118D0A09008038872232220800C0382A
:10056000872232220800AE010030AB222E08303E36
:1005700037229622AE0A2E1EB62A08000030AB2281
:10058000AE01AE0A2E08172096222E1EC12A0800A0
:100590000030AF22AE01AE0A2E08052096222E1E94
:1005A000CB2A080010089020AF002F0890001008F8
:1005B0003002031900001008B00007309005100841
:1005C000ED22900D100AAB220630962207309622BB
:1005D000AF1F0800233096220800AE00703087223B
:1005E0002E08031D142B0330962207309622063066
:1005F0009622063096220630962206309622073042
:100600009622033096221C3096221E309622063007
:1006100096220030962200309622063096221E3016
:1006200096221C3096220800AE03031D382B0F3093
:100630009622073096220630962206309622063001
:10064000962206309622073096220F3096221830D6
:1006500096221C3096220E309622063096220630C4
:1006600096220E3096221C309622183096220800D0
:10067000AE03031D5C2B0F3096220F3096220C30F8
:1006800096220F3096220F3096220C3096220F3091
:1006900096220F3096221E3096221E30962200306F
:1006A00096221C3096221C309622003096221E3054
:1006B00096221E3096220800AE03031D802B0730C1
:1006C000962207309622063096220730962207306F
:1006D00096220630962206309622063096221E304A
:1006E00096221E309622003096221C3096221C3014
:1006F0009622003096220030962200309622080082
:10070000AE03031DA42B073096220F3096220C3027
:1007100096220C3096220C3096220C3096220F3006
:100720009622073096221E3096221E3096220030E6
:1007300096221E3096221E309622063096221E30B9
:1007400096221E3096220800AE03031DC82B0330EC
:1007500096220730962206309622073096220730DE
:1007600096220630962206309622063096221C30BB
:1007700096221E309622063096221E3096221E3079
:1007800096220630962206309622063096220800DF
:10079000073096220730962206309622073096229E
:1007A000073096220630962207309622073096228E
:1007B0001C3096221E309622063096221C3096223D
:1007C0001E309622063096221E3096221C3096222B
:0207D00008001F
:02400E00F13F80
:104200001F001000100010001000100010001F0010
:104210001F000100010001000100010001001F005A
:104220000000080004000200010002000400080071
:104230000000020004000800100008000400020052
:10424000000018001C001E001F001E001C001800AB
:104250000000030007000F001F000F00070003000D
:10426000740068006500470049004D004D0049009A
:1042700043004B002000760030002E00390067001C
:00000001FF
